:100000000C943E000C9450000C9450000C94500042
:100010000C9450000C9450000C9450000C94500020
:100020000C9450000C9450000C9450000C94500010
:100030000C9450000C9450000C9450000C94500000
:100040000C9450000C9450000C9450000C945000F0
:100050000C9450000C9450000C9450000C945000E0
:100060000C9450000C9450000C9450000C945000D0
:100070000C9450000C9450000C94500011241FBE9E
:10008000CFEFCDBFDFE3DEBF28E3A0E0B8E301C0E0
:100090001D92A330B207E1F70E9452000C94CB00EE
:1000A0000C94000082E08093210484E0809321047A
:1000B00088E0809321048091140488608093140464
:1000C00081E08093400680914206806180934206E1
:1000D0008091420687608093420690910238E091B9
:1000E0000038F091013820E030E052E064E048E070
:1000F00076E08091080484FF17C050932604609333
:1001000026042115310531F5409326048091080419
:1001100084FF0AC05093260460932604409326046B
:100120008091080484FDF6CF911509F150932504C0
:10013000409326049F5FE917F10588F46093250436
:100140008091080484FFF2CF509326046093260424
:1001500020E137E22150310940932504CACF609352
:1001600026048091080484FDEFCF9111DFCF7093B6
:1001700046068091480681608093480680914B0630
:1001800080FFFCCFE0915006F0915106F695E7957F
:0A019000F695E795CBCFF894FFCF6A
:00000001FF
